:020000040800F2
:10000000000001207D050008000000000000000045
:1000100000000000000000000000000000000000E0
:1000200000000000000000000000000000000000D0
:1000300000000000000000000000000000000000C0
:1000400000000000000000000000000000000000B0
:1000500000000000000000000000000000000000A0
:100060000000000000000000000000000000000090
:100070000000000000000000000000000000000080
:100080000000000000000000000000000000000070
:100090000000000000000000000000000000000060
:1000A0000000000000000000000000000000000050
:1000B0001D15000800000000000000000000000006
:1000C0000000000000000000000000000000000030
:1000D0000000000000000000000000000000000020
:1000E0000000000000000000000000000000000010
:1000F0000000000000000000000000000000000000
:1001000000000000000000000000000000000000EF
:1001100000000000000000000000000000000000DF
:1001200000000000000000000000000000000000CF
:1001300000000000000000000000000000000000BF
:1001400000000000000000000000000000000000AF
:10015000000000000000000000000000000000009F
:10016000000000000000000000000000000000008F
:10017000000000000000000000000000000000007F
:10018000000000000000000000000000000000006F
:10019000000000000000000000000000000000005F
:1001A000000000000000000000000000000000004F
:1001B000000000000000000000000000000000003F
:1001C000000000000000000000000000000000002F
:1001D000000000000000000000000000000000001F
:0401E0005FF8E0F1F3
:1001E40010B500220A2300F0C9F810BD10B5002193
:1001F4000A2200F06BF910BD41EA0003844613F0B3
:10020400030F10B418BF04460FD10446084609680A
:1002140003E044F8041B50F8041FCB43A1F101325E
:10022400134013F0803FF4D0014600228B5CA354AA
:100234000132002BFAD1604610BC704710F0030F56
:10024400014618BF00460BD108460B6801E050F880
:10025400043FA3F10132DB431A4012F0803FF6D091
:1002640003781BB110F8013F002BFBD1401A7047F3
:1002740070B404461046F2B141EA040313F0030FCC
:100284001ED1032A25460E4618D922680B689A42C5
:100294000FD013E0A2F10133D243134013F0803F97
:1002A40009D10435043603281DD92A6833689A42D3
:1002B40004D10438EED1002070BC70472C4631467E
:1002C400421E23780878984213D1002AF3D00028DC
:1002D400F1D014F8013F11F8010F984209D112F13D
:1002E400FF32F4D1E7E72C4631460028E8D12B78D9
:1002F4003078181AE0E7C04630B4154641EA0002E7
:10030400844612F0030F14BF00230123032D94BF6E
:10031400002303F00103002B2DD004460846016896
:10032400CB43A1F10132134013F0803F05D1043DCA
:100334000430032D44F8041BF1D822460446BDB111
:1003440023781146681E01F8013B53B1023278B19B
:1003540014F8013F1146013802F8013C0132002B28
:10036400F5D128B100231A46CA5401339842FBD16F
:10037400604630BC704702460C46E0E72DE9F04F7A
:100384001F4640F21C0385B0C2F200030E460390E0
:10039400D3F800900291019216F8015B09EB050273
:1003A400537813F00803F7D12D2D04BF4FF0010B40
:1003B40016F8015B04D02B2D9B4608BF16F8015B91
:1003C400D7F1010138BF0021102F14BF0B4641F0B3
:1003D400010343B1302D68D029B1302D02D00A2752
:1003E400B84601E00827B846BBF1000F414614BFE8
:1003F4004FF000446FF00044204600F0B1F820466E
:100404008A46414600F070F804460020014609EB94
:1004140005035B7813F0040F18BFA5F1300208D16F
:1004240013F0030F23D013F0010F14BF3723572306
:10043400EA1A97421BDDA04294BF0023012353EA2A
:10044400D1730FD15245D4BF00230123A04214BF5E
:10045400002303F001032BB908FB0020012116F847
:10046400015BD4E74FF0FF3116F8015BCFE7B1F140
:10047400FF3F0FD0BBF1000F0AD1019B1BB129B97B
:100484000299019A116005B0BDE8F08F711EF8E77A
:100494004042F2E7039ABBF1000F14BF4FF0004053
:1004A4006FF0004022231360E7E73278582A14BF24
:1004B40000230123782A08BF43F00103002B8BD0CB
:1004C40010277578B84602368EE7C046134640F2C8
:1004D4002002C2F2000270B504460D46106821469F
:1004E4002A46FFF74BFF70BD002934D001230022B8
:1004F40010B488422CD301242407A14204D281429F
:1005040002D209011B01F8E7E400A14204D28142AE
:1005140002D249005B00F8E7884201D3401A1A432B
:100524004C08A04202D3001B5C0822438C08A04262
:1005340002D3001B9C082243CC08A04202D3001B18
:10054400DC082243002803D01B0901D00909E3E792
:10055400101C10BC704708B14FF0FF3000F00AB80F
:100564000029F8D003B5FFF7C1FF0EBC4243891A36
:100574001847C0467047C046684620F007018D46BC
:1005840001B540F20002C2F2000240F21413C2F2BA
:1005940000039A4216D24FF0000240F20001C2F268
:1005A400000141F6D82EC0F6000E40F21410C2F23B
:1005B40000005EF802308B5002F1040201EB0203EA
:1005C4008342F6D340F21412C2F2000240F24813FE
:1005D400C2F200039A420DD240F21413C2F2000395
:1005E4004FF0000140F24812C2F2000243F8041B2B
:1005F4009342FBD300F00CFABDE8014085467047F6
:1006040010B44FF0000C614664460BE0D15003F186
:100614000403402BFAD10CF1010C00F14000BCF1B1
:100624003F0F02D002460B46F0E710BC7047C046AD
:1006340070B40D4604464FF0000006460DE05CF829
:1006440002308B5002F10402402AF8D104F1400434
:1006540000F14000B0F57C6F04D005EB0001A44626
:100664003246ECE770BC704782B00190019B33B115
:10067400019B03F1FF330193019B002BF8D102B0DE
:100684007047C04600B583B04FF000604FF00001E2
:1006940000F034FF4FF01C038DF80430A3F11C0369
:1006A4008DF8053003F101038DF806308DF807301D
:1006B40001A800F0DFFE03B000BDC04610B540F253
:1006C4003411C2F200014FF4E1230B60A3F5E123DE
:1006D4008B80CB800B818B814FF00C034B8143F6D5
:1006E4000004C4F20104204601F034F820464FF01F
:1006F400010101F00DF810BD70B540F21811C2F2FD
:1007040000014FF0FF338B804FF000040C80CC804D
:100714004C804FF0804000F02BFF4FF080404FF4AE
:10072400E1514FF0010200F0CBFF40F22211C2F27E
:1007340000010C804FF001054D8040F20003C2F22D
:1007440000031B88CB800C814FF0804000F03AFFFF
:100754004FF08040214600F0B7FF4FF080404FF04B
:1007640002012A4600F09CFF4FF08040294600F029
:1007740087FF70BD30B583B040F6BA23ADF80430BE
:100784004FF010038DF807304FF003048DF8064046
:1007940001AD41F20040C4F20100294600F0F4FD2D
:1007A4004FF40073ADF804308DF806404FF0180391
:1007B4008DF8073040F60004C4F2010420462946AF
:1007C40000F0E2FD4FF48063ADF804304FF0040311
:1007D4008DF807302046294600F0D6FD03B030BD21
:1007E40010B500F075FC4FF4803000F095FC4FF02C
:1007F4003104204600F0AAFD0028FAD04FF0100082
:1008040000F058FC4FF0020000F048FC4FF00000EC
:1008140000F0D0FC4FF0000000F0E4FC4FF48060E6
:1008240000F0D4FC4FF480304FF4801100F09AFCB7
:100834004FF0010000F0A4FC4FF03904204600F012
:1008440085FD0028FAD04FF0020000F09FFC00F074
:10085400A9FC0828FBD144F225004FF0010100F067
:1008640049FD4FF00100014600F05AFD10BDC0469D
:100874002DE9F04F8DB00590049301EBD1734FEA4D
:100884006303069303F1FF33089301FB02F101EBC9
:10089400D1714FEA610107914FF0000B41F200431F
:1008A400C4F201039846039308994FEAC1110291D7
:1008B400089A4FEA420303F101034FEA8313034406
:1008C40001934746049B012B04D103984FF4006124
:1008D40000F0C8FD0899002961DB0599029B01EB32
:1008E40003024FEA8B031A440A92019A13440B93AE
:1008F4004FF0000309930A990E680B9A15684FF09C
:1009040000044FF0800A099B4FEA0319A34505D15F
:1009140038464FF0020100F0A3FD04E038464FF0E2
:10092400020100F09FFD16F0010F19BF0821C8F85D
:1009340010100822C8F8142015F0010F19BF202345
:10094400C8F810302021C8F814103846514600F079
:1009540087FD3846514600F085FD04EB0903079AEC
:10096400934204D138464FF4006100F079FD04F15C
:100974000104102C04D04FEA56064FEA5505C5E78A
:10098400099B03F1010309930A99A1F180010A91DA
:100994000B9AA2F180020B9206998B42ABD1039879
:1009A4004FF4007100F05EFD03984FF4007100F005
:1009B40057FD4FF03200FFF757FE0BF1010BBBF16F
:1009C400100F7FF47FAF0DB0BDE8F08F2DE9F04735
:1009D40007460178C9B14FF0000443F600084546C4
:1009E400C4F201054FF08006C14649B2284689B2D7
:1009F40000F09EFE2846314600F0A6FE0028F9D0FD
:100A040004F10104395D0029EFD1BDE8F087C04647
:100A14002DE9F04FADF5025D8FB0FFF7E1FEFFF772
:100A240031FEFFF7A7FEFFF767FEFFF747FE40F230
:100A34004413C2F200034FF000051D600DF5845409
:100A440004F138042046FFF7DBFD20462EA9FFF70A
:100A5400EFFD02954FF008064FF004010391049650
:100A64004FF00109C84605954FF01402069207920B
:100A7400CDF8209009950A950B920C92CDF83490FC
:100A8400AB462EAFA7F178072EABA3F17E030193FB
:100A94009A4607F10601009141F20044C4F20104B0
:100AA40020464FF0100100F0D5FCC0F101022046B1
:100AB4004FF01001D2B200F0D7FC43F60000C4F2AC
:100AC40001004FF0200100F03FFE012840F02A828F
:100AD40043F60000C4F2010000F030FE00F07F0095
:100AE400785540B2292818BF013540F01B8207EB26
:100AF40005024FF000035370384641F63021C0F62A
:100B040000014FF00302FFF7B3FB40B941F6342074
:100B1400C0F60000FFF75AFF4FF0000502E2384626
:100B240041F64021C0F600014FF00302FFF7A0FB9D
:100B340040B941F64420C0F60000FFF747FF4FF0EC
:100B44000005EFE1384641F66421C0F600014FF09C
:100B54000902FFF78DFBD0B9384607F10A01FFF708
:100B64004BFB504639464FF00202FFF7C5FB4FF0EE
:100B74000004019A94705046FFF738FB039041F645
:100B84007020C0F60000FFF721FF2546CAE1384671
:100B940041F67421C0F600014FF00902FFF768FB2B
:100BA400D0B9384607F10A01FFF726FB504639460B
:100BB4004FF00202FFF7A0FB4FF00004019B9C7072
:100BC4005046FFF713FB049041F67020C0F6000076
:100BD400FFF7FCFE2546A5E1384641F68021C0F624
:100BE40000014FF00902FFF743FB00286AD13846A1
:100BF40007F10A01FFF700FB504639464FF00302A4
:100C0400FFF77AFB019991F900304F2B1CBF0022AA
:100C1400099207D1019991F901304E2B14BF002399
:100C240001230993384607F10401FFF7E5FA50461A
:100C340039464FF00502FFF75FFB4FF00004019ABD
:100C440054715046FFF7D2FA80B240F20003C2F268
:100C54000003188038460099FFF7CEFA504639460B
:100C64004FF00502FFF748FB019B5C715046FFF70C
:100C7400BDFA069038460099FFF7BEFA5046394649
:100C84004FF00502FFF738FB01994C715046FFF70E
:100C9400ADFA079038460099FFF7AEFA5046394648
:100CA4004FF00502FFF728FB019A54715046FFF7F5
:100CB4009DFA089041F67020C0F60000FFF786FE0A
:100CC40025462FE1384641F68C21C0F600014FF04D
:100CD4000802FFF7CDFA00286BD1384607F1090165
:100CE400FFF78AFA504639464FF00302FFF704FB38
:100CF400019991F900304F2B18BF4FF0000B08D128
:100D0400019A92F901304E2B14BF4FF0000B4FF0B3
:100D1400010B384607F10401FFF76EFA50463946D5
:100D24004FF00502FFF7E8FA4FF00004019B5C71F5
:100D34005046FFF75BFA80B240F20003C2F20003B0
:100D4400188038460099FFF757FA504639464FF055
:100D54000502FFF7D1FA01994C715046FFF746FAA4
:100D64000B9038460099FFF747FA504639464FF042
:100D74000502FFF7C1FA019A54715046FFF736FA9B
:100D84000C9038460099FFF737FA504639464FF031
:100D94000502FFF7B1FA019B5C715046FFF726FA92
:100DA4000D9041F67020C0F60000FFF70FFE2546B7
:100DB400B8E0384641F69821C0F600014FF0080229
:100DC400FFF756FA002838D1384607F10901FFF732
:100DD40013FA02994FEA81120DF5845303F1380393
:100DE40003EB02044FF005054FF000060FE05046F8
:100DF40039462A46FFF780FA019A56715046FFF7A2
:100E0400F5F944F8040C38460099FFF7F5F938462B
:100E1400FFF714FA04F104040528E8D8029B03F14F
:100E24000103029341F67020C0F60000FFF7CEFDE7
:100E3400029E4FF00005A84674E0384641F6A4210E
:100E4400C0F600014FF00702FFF712FA90B90DF552
:100E5400845000F138002EA9FFF7EAFB41F6702018
:100E6400C0F60000FFF7B2FD4FF0000502954FF009
:100E7400010857E0384641F6AC21C0F600014FF0B6
:100E84000502FFF7F5F918BB0DF5845404F1380495
:100E94002046FFF7B5FB2EAD20462946FFF7C8FBD9
:100EA40028460399049A4FF00103FFF7E1FC41F649
:100EB4007020C0F60000FFF789FD4FF00005029591
:100EC4004FF00109A846059509950A95AB4629E016
:100ED400384641F6B421C0F600014FF00A02FFF78C
:100EE400C7F9A0B9B8F1000F08D041F6C020C0F688
:100EF4000000FFF76BFD4FF0000513E041F6C8203A
:100F0400C0F60000FFF762FD4FF000050AE041F66D
:100F1400D020C0F60000FFF759FD3846FFF756FD14
:100F24004FF00005B8F1000F3FF4B6AD2EA80399B9
:100F3400049A4B46FFF79CFCBBF1000F34D00C9A8B
:100F44000B9902EB01030A9999420FDD0D9AB2F154
:100F5400FF3F12D002F1FF320D92002ADEBF4FF0A4
:100F64000008CDF82880C34607DC0BE00A9B0B99E8
:100F74008B4208BF4FF0000904E04FF001094FF025
:100F840000020A9240F24413C2F200031B68012BD0
:100F94000AD140F24413C2F200034FF000021A6077
:100FA4000A9B03F101030A93099900293FF474ADE4
:100FB4000799069A01EB02034FEA06121344059AB5
:100FC4009A4225DD089BB3F1FF3F0AD10DF5845009
:100FD40000F138002EA9FFF72BFB4FF0000105911B
:100FE40016E0089A02F1FF320892002ADEBF4FF0A1
:100FF4000008CDF81480CDF8248009DD0DF5845067
:1010040000F138002EA9FFF713FB4FF000030593FE
:1010140040F24413C2F200031B68012B7FF43CAD81
:1010240040F24413C2F200034FF000021A60059923
:1010340001F101010591069A8A42BFBF00210846C9
:101044002EAC06F1FF3EB8BF84461DDB24E54FEA13
:101054000113034454F823204FEA420244F82320A6
:1010640071450FDA01F101034FEA0313034454F805
:10107400233013F4004F1FBF0B011B1842F0010271
:1010840044F8232001F10101B142E0DB00F1010049
:101094000F283FF701AD6146F6E7C04642F2000370
:1010A400C4F202031A6802F0380240EA020018602F
:1010B4007047C04642F20002C4F20202136823F0F1
:1010C40010031360136840EA030010607047C046C1
:1010D40041F20001C4F202010B6843F001030B600A
:1010E4004A6840F20003CFF6FF0302EA03024A60B3
:1010F4000A684FF6FF73CFF6F66302EA03020A604A
:101104000B6823F480230B604B6823F4FE034B60CD
:101114004FF41F038B60704741F20003C4F20203D3
:101124001A6822F480321A601A6822F480221A6043
:10113400B0F5803F03D0B0F5802F11D108E041F223
:101144000002C4F20202136843F48033136007E020
:1011540041F20002C4F20202136843F4A0231360B4
:101164007047C04641F20003C4F202035A6822F4F5
:101174007C1240EA020040EA010058607047C04611
:1011840040F26003C4F242231860704741F2000346
:10119400C4F202035A6822F0030240EA02005860D3
:1011A4007047C04641F20003C4F20203586800F0DD
:1011B4000C00704741F20003C4F202035A6822F0A3
:1011C400F00240EA020058607047C04641F2000352
:1011D400C4F202035A6822F4E06240EA0200586052
:1011E4007047C04641F20002C4F20202536823F47D
:1011F400605343EAC00353607047C04610B40446CA
:1012040041F20003C4F202035B6803F00C03042BF5
:1012140002BF41F60033C0F2B70303603AD0082B93
:1012240007D0002B31D141F20023C0F27A030360CE
:1012340030E041F20003C4F202035A685B6802F42E
:1012440070124FEA924202F1020213F4803F01BF8E
:1012540040F60013C0F23D03534303601AD041F239
:101264000003C4F202035B6813F4003F1FBF48F697
:101274008053C0F25B035343036001BF41F6003364
:10128400C0F2B7035343036004E041F20023C0F209
:101294007A03036041F20000C4F20200436803F0E1
:1012A400F0034FEA131340F20201C2F20001CB5CD7
:1012B400226822FA03F26260436803F4E0634FEAAF
:1012C4001323CB5C22FA03F3A360436803F4605353
:1012D4004FEAD323CB5C22FA03F2E260436803F4BF
:1012E400404301EB93310B7CB2FBF3F2226110BC5F
:1012F4007047C04641B141F20002C4F20202936950
:1013040040EA0303936109E041F20003C4F20203DB
:1013140099696FEA000202EA01029A617047C046C5
:1013240041B141F20002C4F20202D36940EA03036C
:10133400D36109E041F20003C4F20203D9696FEA00
:10134400000202EA0102DA617047C0464FEA501314
:10135400012B02BF41F20003C4F202031B680CD04C
:10136400022B03BF41F20003C4F202031B6A41F2E1
:1013740000031CBFC4F202035B6A00F01F0023FADF
:1013840000F000F0010070472DE9F003064608461E
:10139400CB7803F00F0713F0100F1CBF8B781F439B
:1013A4000B783BB334684FF0000C4FF001054FF05D
:1013B4000F0805FA0CF2038802EA0301914213D1E3
:1013C4004FEA8C0208FA02F36FEA030303EA040308
:1013D40007FA02F243EA0204C378282B08BF7161BA
:1013E40002D0482B08BF31610CF1010CBCF1080F8D
:1013F400DFD134600388FF2B29D975684FF0000CC6
:101404004FF001084FF00F090CF1080308FA03F13B
:10141400038801EA03048C4213D14FEA8C0309FACE
:1014240003F26FEA020202EA050207FA03F342EA50
:101434000305C378282B08BF7461C378482B08BF01
:1014440031610CF1010CBCF1080FDDD17560BDE810
:10145400F0037047C36819420CBF00200120704795
:1014640001617047416170470AB1016100E0416167
:101474007047C046C3787BB34EF60053CEF20003E8
:10148400DB686FEA030303F4E0634FEA1323C3F159
:101494000402417801FA02F14FF00F0222FA03F23A
:1014A400837802EA030242EA010200784FEA021258
:1014B400D2B24EF20011CEF2000101EB000383F828
:1014C40000234FEA501200F01F004FF0010303FA0B
:1014D40000F341F8223010E003784FEA531103F08F
:1014E4001F034FF0010202FA03F24EF20013CEF290
:1014F400000301F1200143F8212070474FF6807367
:10150400C1F6FF7301EA030141EA00014EF60053FC
:10151400CEF200039960704710B54FF080404FF051
:10152400020100F0E3F808B34FF080404FF00201ED
:1015340000F0E8F840F24413C2F200034FF0010255
:101544001A604FF0804000F0CDF840F21413C2F25C
:101554000003188040F20003C2F200031B8800EB72
:1015640003014FF0804089B200F0BAF810BDC046C4
:10157400038803F08F03038003889BB2CA8843EA7D
:1015840002034A8843EA02039BB203808B88838563
:101594000B88038542F60042C4F2010243F2004381
:1015A400C4F20103984214BF00230123904208BFF0
:1015B40043F001030BB10B7A03864FF001038382DE
:1015C4007047C046F0B40C46038C23F001034FEA85
:1015D40003434FEA13430384018C83889DB2038B36
:1015E4009EB2278821F002014FEA01414FEA1141DE
:1015F4006388228943EA02039BB243EA010C42F660
:101604000042C4F2010243F20043C4F201039842CF
:1016140014BF00230123904208BF43F00103F3B138
:101624004FF6F773C0F200030CEA0303628943EA3E
:1016340002034FF6FB72C0F2000203EA0202A3881F
:1016440042EA030C47F6FF41C0F2000105EA01013A
:10165400E389A28943EA02039BB243EA0105858038
:101664004FF68C73C0F2000306EA030343EA070350
:101674000383E3888386A0F820C0F0BC7047C0468B
:1016840029B103889BB243F00103038007E0038878
:1016940023F001034FEA83534FEA935303807047C7
:1016A4002AB183899BB241EA0303838106E08389DB
:1016B4009BB26FEA010203EA020383817047C046CA
:1016C400018582827047C046038B23F008034FEAEA
:1016D40003434FEA134341EA030101837047C046C1
:1016E40081867047808E80B27047C046038A8289A3
:1016F40019420CBF0020012011420CBF002000F051
:10170400010070476FEA010189B201827047C04647
:1017140029B183899BB243F40053838107E0838911
:1017240023F400534FEA03434FEA13438381704782
:101734004FEAC1514FEAD1518180704780884FEA06
:10174400C0504FEAD0507047038819420CBF0020A4
:101754000120704730B587B005460C46038A23F450
:1017640040534FEA03434FEA1343CA8843EA020350
:101774000382828922F4B05222F00C024FEA024220
:101784004FEA12420B89898843EA0103618943EADB
:1017940001039BB243EA02038381838A23F44073E7
:1017A4004FEA03434FEA1343A28943EA02038382C5
:1017B40001A8FFF723FD43F60003C4F201039D4291
:1017C4000CBF049903994FEAC1024FEA4113C2EBDB
:1017D40003030B4422684FEA8202B3FBF2F348F29C
:1017E4001F54C5F2EB14A4FB03204FEA50104FEA38
:1017F40000104FEA10124FEA82014FEA021211441C
:101804004FEA81021144C1EB03034FEA031303F1CE
:101814003203A4FB03234FEA531303F00F0343EAF9
:1018240000039BB22B8107B030BDC04630B587B0F2
:1018340044F205004FF00101FFF75CFD4FF48040D6
:101844004FF00101FFF756FD4FF40073ADF814306B
:101854004FF003038DF8163003F115038DF817309C
:1018640040F60004C4F2010405AD20462946FFF702
:101874008BFD4FF48063ADF814304FF004038DF802
:10188400173020462946FFF77FFD4FF41653019386
:10189400A3F51653ADF80830ADF80A30ADF80C30A6
:1018A400ADF810304FF00C03ADF80E3043F60004E1
:1018B400C4F20104204601A9FFF74CFF20464FF073
:1018C4000101FFF725FF40F21613C2F200034FF0A7
:1018D40001021A7007B030BD70B5064640F2161307
:1018E400C2F200031B780BB9FFF7A0FF0A2E03D145
:1018F4004FF00D00FFF7F0FF43F600031D46C4F25E
:1019040001054FF0800428462146FFF71DFF0028FB
:10191400F9D043F60000C4F20100F1B2FFF708FF6A
:1019240070BDC046101C70470020202020202020BD
:10193400202028282828282020202020202020207B
:10194400202020202020202020881010101010108B
:1019540010101010101010101004040404040404D7
:101964000404041010101010101041414141414171
:101974000101010101010101010101010101010153
:101984000101010110101010101042424242424263
:101994000202020202020202020202020202020223
:1019A40002020202101010102000000000000000CB
:1019B4000000000000000000000000000000000023
:1019C4000000000000000000000000000000000013
:1019D4000000000000000000000000000000000003
:1019E40000000000000000000000000000000000F3
:1019F40000000000000000000000000000000000E3
:101A040000000000000000000000000000000000D2
:101A140000000000000000000000000000000000C2
:101A240000000000000000000000000057686F0084
:101A34004F4B3A4C45445369676E0000566572003B
:101A44004F4B3A48617264205665723D302E312CFA
:101A5400204669726D205665723D302E31000000BB
:101A64005365744C4544436E740000004F4B0000B2
:101A74005365744272696768740000005365745357
:101A840063726F6C6C000000536574426C696E6B1A
:101A9400000000005365744C436F6465000000004F
:101AA400446973706C617900436C65617200000075
:101AB400526561645374617475730000427573797F
:101AC4000000000049646C65000000004E473A00C5
:041AD40043000000CB
:101AD800F4010000000001020304010203040607E8
:101AE80008090204060800002D1900082C1900082E
:101AF800240000200000000000000000000000009A
:101B080000000000000000000000000000000000CD
:101B180000000000D41A00080000000000000000C7
:101B280000000000000000000000000000000000AD
:101B3800000000000000000000000000000000009D
:101B4800000000000000000000000000000000008D
:101B5800000000000000000000000000000000007D
:101B6800000000000000000000000000000000006D
:101B7800000000000000000000000000000000005D
:101B8800000000000000000000000000000000004D
:101B9800000000000000000000000000000000003D
:101BA800000000000000000000000000000000002D
:101BB800000000000000000000000000000000001D
:101BC800000000000000000000000000000000000D
:101BD80000000000000000000000000000000000FD
:041BE80000000000F9
:04000005080001E40A
:00000001FF
